:10000000112484B714BE81FF22D185E08EBD8EE01D
:100010001AD1D49AD29A86E023EC3FEF91E03DBD0D
:100020002CBD9BB9589BFECFCC9AA8958150B9F7AF
:10003000DD24D39485E0C82E0FE7F02E1EECE12ED0
:10004000E9D0813421F481E00DD183E020C08234F5
:1000500011F484E103C0853419F485E003D1C8C0EC
:10006000853581F4D7D0082F10E0D4D090E0982FB8
:100070008827802B912B880F991F90938101809363
:100080008001B5C0863529F484E0ECD080E0B3D09F
:10009000AFC0843609F06BC0D1D0C0E0D1E0BAD097
:1000A0008993809182018150809382018823B9F7DE
:1000B000E0918001F091810183E087BFE895CCD089
:1000C00007B600FCFDCF8091800190918101892BC2
:1000D00041F5809100012091010130E0322F22276B
:1000E00090E0282B392B3093850120938401409197
:1000F00008018091090190E0982F882750E0842B17
:10010000952B909387018093860124503040209353
:100110000801232F332720930901F0920001E09278
:1001200001014091800150918101A0E0B1E02C914A
:1001300030E011968C91119790E0982F8827822BB0
:10014000932B1296FA010C01D7BEE89511244E5F4D
:100150005F4FF1E0A034BF0751F7E0918001F091CB
:100160008101C7BEE89507B600FCFDCF41C08437CA
:1001700089F564D071D0E0918001F09181013097D0
:1001800019F42091840113C0E130F10519F4209194
:1001900085010DC0E830F10519F42091860107C0F2
:1001A000E930F10519F42091870101C02491809173
:1001B000800190918101019690938101809380014B
:1001C000822F19D0809182018150809382018823EF
:1001D00091F60EC0853739F43FD08EE10CD083E91B
:1001E0000AD08CE054CF813511F488E02CD034D083
:1001F00080E101D025CF2AE030E08095089410F40A
:10020000DA9802C0DA9A000015D014D086952A95A3
:10021000B1F70895A89529E030E0CB99FECF0AD038
:1002200009D008D08894CB9908942A9511F0879525
:10023000F7CF08959EE09A95F1F70895EBDFEADF96
:1002400080938201E7CF98E191BD81BD089580E060
:10025000FADFE4E0FF270994DDDF803209F0F7DF01
:1002600084E1C9CF1F93182FD5DF1150E9F7F4DFD0
:040270001F9108953D
:021EFE000104DD
:00000001FF
